:03000000020100FA
:0100030032CA
:0100130032BA
:01001B0032B2
:04002300120E69321E
:03004B00C2D132ED
:01005300327A
:01005B003272
:01006300326A
:01006B003262
:100080002A202A202A2053796E747261636B202AF9
:100090002050726F6772616D6D6564206279204DCA
:1000A00061726B7573204D6569657220666F722091
:1000B000537065637472616C20417564696F2028A8
:0D00C00063292031393937202A202A202ACF
:1001000000758780758922758DFE758BFEC2DFD2E2
:100110008E75985075810F754500C27FC27E7544FB
:1001200000C27CC27DC27AD26CC27BC279C27675B3
:100130004700D274D273D278D277D272D263D264AB
:10014000756B007880760078817602788276007808
:10015000837602754800754900754380756A01C24F
:10016000D3C2D4754600C2DB755401C26D756600FA
:10017000D26A7542007540007562A17563A079006E
:100180007A087830120D6A53300FC244120CC3E55E
:1001900037A2E09268A2E19267A2E2926675A91086
:1001A00075B910D2ACC2CDD2AFA278B074400FA254
:1001B00078B3B074B079B07650024173418B207936
:1001C0001D30760241610531E531B463037531625A
:1001D000120CC3755F02120E38754800418BE5475B
:1001E000B400110530E530B4100375300F754400CC
:1001F000D26C418BB401181532E532B40B03753261
:1002000006B40503753204B40003753201807CB472
:10021000021015341534E534C3940A500375340ABA
:100220008069B403181536E536B40B03753606B489
:100230000503753604B40003753601804EB404041A
:10024000D2688047B4050C0535E535B4040375352F
:10025000038038B40604D2678031B4072ED266809A
:100260002A0538E538B46403753880B4E40375387A
:10027000E38018E548B4FF130531E531B463037535
:100280003162120CC3755F02120E380548A27492D7
:1002900078A277B073400FA277B3B073B079B0761D
:1002A0005002615B617320791D307602614915311E
:1002B000E531B4FF03753100120CC3755F02120EF5
:1002C000387549006173E547B400111530E530B465
:1002D000FF03753000754400D26C6173B4011805DA
:1002E00032E532B40503753206B4070375320CB437
:1002F0000D0375320C807CB4021005340534E534EE
:10030000C394CE40037534CD8069B403180536E537
:1003100036B40503753606B4070375360CB40D0301
:1003200075360C804EB40404C2688047B4050C15C1
:1003300035E535B4FF037535008038B40604C2676F
:100340008031B4072EC266802A1538E538B4FF0321
:10035000753800B47F037538638018E549B4FF131E
:100360001531E531B4FF03753100120CC3755F021E
:10037000120E380549A273927720795B207619E531
:10038000310475F00A84120C7E8829E5F0120C7E87
:10039000882AA26C9257A13F054AE54AB4FF05B2EC
:1003A00075754A002075087529FF752AFFA13FE57C
:1003B00038D2D530E704C2E7C2D575F00A84120CF2
:1003C0007E8829A2D5924FE5F0120C7E206C04E8BD
:1003D000C2E7F8882AA13FE547B40239054AE54A51
:1003E000B4FF05B275754A0020750C7529AF752AE2
:1003F000FFA26C9257A13FE534F4C313C394187560
:10040000F00A84120C7E8829E5F0120C7E882AA25C
:100410006C9257A13FE547B4001CE5300475F00A23
:10042000847529A7B40102C24FE5F0120C7E882A18
:10043000A26C9257A13FB40158E532B4011075295E
:100440000C7402120C7E882AA26C9257A13FB4024F
:10045000097406120C7E882A802EB40309740412D3
:100460000C7E882A8022B404097403120C7E882A28
:0E0470008016B406097402120C7E882A800AD7
:10047E00B40C077401120C7E882A75298CA26C921A
:10048E0057A13FB40358E536B40110752921740203
:10049E00120C7E882AA26C9257A13FB402097406F0
:1004AE00120C7E882A802EB403097404120C7E88E6
:1004BE002A8022B404097403120C7E882A8016B492
:1004CE0006097402120C7E882A800AB40C07740185
:1004DE00120C7E882A7529A1A26C9257A13FB404F2
:1004EE00137529C7E4A26892E0120C7E882AA26CCA
:1004FE009257A13FB40510752986E535120C7E88FA
:10050E002AA26C9257A13FB4061375298EE4A267F6
:10051E0092E0120C7E882AA26C9257A13FB407116A
:10052E00752987E4A26692E0120C7E882AA26C924C
:10053E0057E554B4011E75E8FFC297D297D2FED28A
:10054E00FFC2FD852AE8C297D297A2B29273A2B3D8
:10055E009274C1DBB4025575E8FFC297D297C2FE02
:10056E00D2FFD2FD8529E8C297D297A2B2401520BC
:10057E007904D276800E206DFD755F00C279120E61
:10058E0038206DFDA2B392D5401C207619B3B072FF
:10059E004014207907D279754700800A0547E54750
:1005AE00B40803754700A2D59272C1DBB403028072
:1005BE0002C1DB75E8FFC297D297D2FEC2FFD2FD11
:1005CE008528E8C297D297A2B292D5401BB3826E0D
:1005DE005016B270755F017560442070057561002C
:1005EE00800375617F120E38A2D5926EA2B392D59A
:1005FE004069B3826F5064307902C1B520765EE5F2
:10060E0031C3941D4055E531C3944040277562A314
:10061E007563A2E531C3944075F007A4F97A0778A3
:10062E0038E53AA27092E0F53A120D98E53AC2E03A
:10063E00F53A80277562A17563A0E531C3941D75E7
:10064E00F007A42409F97A077838E53AA27092E007
:10065E00F53A120D98E53AC2E0F53A806CE531C3F1
:10066E00941D5004C2768061E531C39440401B75E1
:10067E0062A37563A2E531C3944075F007A4F97ABD
:10068E00017838120D98C276803F7562A17563A00D
:10069E00E531C3941D75F007A42409F97A01783861
:1006AE00120D98C2768022C279E4A26892E0A26707
:1006BE0092E1A26692E2F5377562A17563A07900A8
:1006CE007A087830120D98C244A2D5926F0554E57F
:1006DE0054B40403755401306109756600C26AC2D0
:1006EE006BC261206A0D1566E566B40004D26AB26B
:1006FE006B80090566E566B53402C26A740C8566C0
:10070E00F0A4C4540FF8E5F0C4F5F0E845F08534D4
:10071E00F0F8E5F0C4F5F0E853F00F8475F00AA494
:10072E00F564C3E556941875F00AA4F54B85F04CA4
:10073E00E5438532F084254BF54B7400354CF54C72
:10074E0074808532F084C54BC3954BF54BE54C94C4
:10075E0000F54CE5648536F084F5F0E5424540C37E
:10076E0013C313C313A4FCE5F0C4FDECC4540F4D26
:10077E0075F00F84C4FBE5F0C4FDEC540F4D75F01D
:10078E000F842B206B11F5F0E54BC395F0F54BE57F
:10079E004C9400F54C800A254BF54BE54C3400F596
:1007AE004CE54CC4FCE54BC4540F4C75F00A84C4A4
:1007BE00F54DE5F0C4FCE54B540F4C75F00A8485FD
:1007CE00F04E254DF54DC333FC75831E8C8274009F
:1007DE0093F54F0582740093F5500582740093C310
:0E07EE00954FFCE54DB42A027C1EEC854EF0C2
:1007FC00A4FCE5F0C4FDECC4540F4D75F00A84C4A0
:10080C00F551E5F0C4FDEC540F4D75F00A842551FB
:10081C00254FF551E5503400F552A26992F765F079
:10082C0030E70BC2C1D2B9D2D120D1FDC2B9E55249
:10083C00A2E792969269C293C2958551E8D29385AC
:10084C0052E8D295A26C92B4306504D2B4C265D28F
:10085C00FBC2B5E546B4004E7400306711E556C3D3
:10086C009423C333F5F0C313C313C31325F0F5F06E
:10087C00E535B4020AE5F02541500274FF8008E525
:10088C00F02539500274FFF5F0E556C3943350113E
:10089C00E556C39423232323247FF995F050028932
:1008AC00F085F0E88059B4010CE53AC3940E500180
:1008BC00E4F5E8804AB40205853BE88042B4030DB8
:1008CC00E53C240B500274FFF4F5E88032B4040FBD
:1008DC00E535B40104E5418002E533F5E88020B448
:1008EC00050FE535B40304E5418002E53DF5E880EC
:1008FC000EB4060BE53E2408500274FFF4F5E8D262
:10090C00B5E546A2E092F8A2E192F9A2E292FAC20F
:10091C00FB0546E546B40703754600E546A2E092A2
:10092C00D8A2E192D9A2E292DA000000000075DAB6
:10093C000020DCFDE5D923235403F5F0901D009332
:10094C00F5DA20DCFDE5D92408F5D9E5F03400F51D
:10095C00F0E546B4000280030209F1E5D97880265F
:10096C00FAE5F078813613F5F0F6EA13F5D97880CC
:10097C00F6E5572403F8E56C3400F9E895D9E995C8
:10098C00F04016E5579404F8E56C9400F9E8C3952B
:10099C00D9E995F05003020C5285D95785F06CE5D6
:1009AC00D9C39408F8E5F09400F5F0E80303A2F03D
:1009BC0092E6A2F192E7F539D240755F01756002BB
:1009CC00E539C31392D5F561120E38206DFD7CF01C
:1009DC00DCFEA2D5E492E6F561756022755F01122A
:1009EC000E38020C52B4015BE5582407F8E56D345F
:1009FC0000F9E895D9E995F04016E5589408F8E522
:100A0C006D9400F9E8C395D9E995F05003020C52A6
:100A1C0085D95885F06DE5D9C39408F8E5F09400B4
:100A2C00F5F0E80303A2F092E6A2F192E7F53AD2D0
:100A3C0041755F01756011E53AC313F561120E380B
:100A4C00020C52B402028003020ADEE5D978822637
:100A5C00FAE5F078833613F5F0F6EA13F5D97882D7
:100A6C00F6E5592403F8E56E3400F9E895D9E995D3
:100A7C00F04016E5599404F8E56E9400F9E8C39536
:100A8C00D9E995F05003020C5285D95985F06EE5E1
:100A9C00D9C39408F8E5F09400F5F0E80303A2F04C
:100AAC0092E6A2F192E7F53BD242755F01756012B6
:100ABC00E53BC31392D5F561120E38206DFD7CF029
:100ACC00DCFEA2D5E492E6F561756032120E3802B6
:100ADC000C52B4035BE55A2407F8E56F3400F9E8CF
:100AEC0095D9E995F04016E55A9408F8E56F94000D
:100AFC00F9E8C395D9E995F05003020C5285D95AFF
:100B0C0085F06FE5D9C39408F8E5F09400F5F0E8AA
:100B1C000303A2F092E6A2F192E7F53CD243755F93
:100B2C0001756013E53CC313F561120E38020C52CB
:100B3C00B4045BE55B2407F8E5703400F9E895D95B
:100B4C00E995F04016E55B9408F8E5709400F9E837
:100B5C00C395D9E995F05003020C5285D95B85F009
:0E0B6C0070E5D9C39408F8E5F09400F5F0E8C0
:100B7A000303A2F092E6A2F192E7F533D244755F3D
:100B8A0001756007E533C313F561120E38020C5282
:100B9A00B4055AE55C2407F8E5713400F9E895D9FB
:100BAA00E995F04016E55C9408F8E5719400F9E8D7
:100BBA00C395D9E995F05003020C5285D95C85F0AA
:100BCA0071E5D9C39408F8E5F09400F5F0E8030359
:100BDA00A2F092E6A2F192E7F53DD245755F017562
:100BEA006014E53DC313F561120E38805BB40658F4
:100BFA00E55D2407F8E5723400F9E895D9E995F03E
:100C0A004016E55D9408F8E5729400F9E8C395D9B1
:100C1A00E995F05003020C5285D95D85F072E5D949
:100C2A00C39408F8E5F09400F5F0E80303A2F09203
:100C3A00E6A2F192E7F53ED246755F01756015E5C9
:100C4A003EC313F561120E38306405120CC3C26438
:100C5A00E56BB49603120CC3056BE56BB498037588
:100C6A006B978538E8C292D292A27092FC7832D8F9
:100C7A00FE0201A9B4000478C0803DB4010478F9E9
:100C8A008036B4020478A4802FB4030478B0802894
:100C9A00B4040478998021B405047892801AB406C1
:100CAA000478828013B4070478F8800CB4080478B6
:100CBA00808005B40902789022E531C3941D404F23
:100CCA00E531C3944040237562A37563A2E531C33D
:100CDA00944075F007A4F97A077838120D6AE53A54
:100CEA00A2E09270C2E0F53A80697562A17563A0CC
:100CFA00E531C3941D75F007A42409F97A077838F9
:100D0A00120D6AE53AA2E09270C2E0F53A8044E533
:100D1A003175F007A4F58275831F740093F53805C1
:100D2A0082740093F5390582740093F53A0582744A
:100D3A000093F53B0582740093F53C058274009399
:100D4A00F53D0582740093F53EE53AA2E09270C241
:100D5A00E0F53AC240C241C242C243C245C246223B
:100D6A00E563120D8C4011E562120DB440F2D271A6
:100D7A00DA09C271120E12F6020DD2120E12F6081A
:100D8A0080EE120DB44006E9120DE740F522E56344
:100D9A00B18C4015E6120DE740F4120DD27B1E7C91
:100DAA0096DCFEDBFA0809DAE5227C03D2B7120EDA
:100DBA000CD2B6120E0CC2B7120E0CC2B6120E0C20
:100DCA00120DE75002DCE522C2B6120E0CC2B712AF
:100DDA000E0CD2B6120E0CD2B730B7EC227F083303
:100DEA0092B700D2B6120E0CC2B6120E0CDFF03356
:100DFA00D2B700D2B6120E0CA2B7C2B6120E0D406E
:100E0A00C722227B06DBFE22D2B7007F08D2B6D1E8
:100E1A000CA2B733C2B6D10CDFF3D2B7D10C307102
:100E2A0002C2B7D10CD2B6D10CC2B680D622206D7E
:100E3A002D7B96DBFEE55FB400057599F08014B44E
:100E4A000108E53044B0F5998009B40211E530444F
:100E5A00C0F599D26D755E0175670075690122C288
:100E6A00ACC0D0C0E0C0F0D2D320980920990302C8
:100E7A0012A40211B6C298859968E56830E75A54F7
:100E8A00F0B4F049E568540FB40007D27F756900E1
:100E9A008038B40704C27F8031B40204D27E802A2B
:100EAA00B40304D27D8023B40F07D26C754400804A
:100EBA0019B40104D27D8012B4080F056AE56AB438
:100ECA000D08756A01306802D2610212A4C4F545A0
:100EDA0085686553650F0212A4307F78E569B4000E
:0E0EEA000BC263E568B47067D2638063B40125
:100EF8000BE568B401028059C2638055306354B46D
:100F08000205856867804AB40327E567A2E0E568BB
:100F180092E7C3940192D5F55EE567C313A2D59411
:100F280000A2E074A192E1F56274A092E1F56380F9
:100F380020B40408E568A2E092628015B40514A202
:100F480062E56892E7F5687868A95E7A01B19880E9
:100F58000205690212A4307D04C27D8025207E2C02
:100F6800E565B5301D207C76E545B4092EE568C3F6
:100F780094234011E568C39461500A856853C27B85
:100F8800D27C0212A4D27BD27C0212A4307C07C28B
:100F98007CC27E0212A4D27C0212A4E545B40B08DE
:100FA80085683FD27C0212A4B40C12E568C394622F
:100FB8004003756862856831D2640212A4B40D06D4
:100FC8008568400212A4B40E05D27C0212A4B408AB
:100FD80005D27C0212A4B40A02D27C0212A4C27CFA
:100FE800E545B4093A307B05C27B0212A4E5686086
:100FF800180544856841E541C333F541306602D29E
:1010080065C26C8553560212A41544E544B4FF0327
:10101800754400207A06E5447002D26C0212A4B42A
:10102800081E307B05C27B0212A41544E544B4FFB8
:1010380003754400207A06E5447002D26C0212A4BB
:10104800B40B0BE53FB401098568420212A40211F2
:1010580093B40216E568238539F0A2F092E0B5F062
:10106800028004F539C2400212A4B422158568F042
:10107800A2F6E53992E0B539028004F539C240029A
:1010880012A4B40714E56823F8E533C313B568025E
:101098008004C24488330212A4B41015E568F4C26F
:1010A800E723F894C4400278C4E82409F53402120E
:1010B800A4B41114E56823F8E53AC313B5680280AF
:1010C80004883AC2410212A4B41216E56823853B8B
:1010D800F0A2F092E0B5F0028004F53BC2420212A1
:1010E800A4B432158568F0A2F6E53B92E0B53B0260
:1010F8008004F53BC2420212A4B41314E56823F835
:10110800E53CC313B568028004883CC2430212A4BC
:10111800B44014E568C39440B3927A207A06E54453
:101128007002D26C0212A4B4440BE568C39440B3B5
:1011380092700212A4B47B0FE568704C75440020CD
:101148007A46D26C0212A4B41414E56823F8E53D7B
:10115800C313B568028004883DC2450212A4B415C1
:1011680014E56823F8E53EC313B568028004883E99
:10117800C2460212A4B41607E568F5380212A4B4F0
:101188001706E568D2E7F5380212A4B40E11E5682F
:1011980023F543C39408400AE543C394F850090271
:1011A80012A47543080212A47543F80212A4C29946
:1011B800E55FB40002800302126A7978D9FEE56916
:1011C800B4001F7B327C96DCFEDBFAE567B4020CC8
:1011D800E55EB40107C26DC2760212687599F00225
:1011E8001266B40106759970021266B40205759903
:1011F80001806BB407087599F77569008062B403BC
:101208000BE55EA2E7E56733F5998052B40408E57B
:101218005EC2E7F5998047E55EC39401F9E56794F6
:1012280000B401087562A37563A280067562A17592
:1012380063A07A017855120D6AE569B4050BE55586
:10124800A2E7E492E0F5998015B40614E555C2E7E3
:10125800F599E55E2401F55EE5673400F5670569F3
:0E126800803AB4011EE55EB4010585609980F0
:1012760006B40203856199055EE55EB40305755EF5
:1012860000C26D8019B40216E55EB401038531997A
:10129600055EE55EB40205755E00C26D8000C2D3D0
:0912A600D0F0D0E0D0D0D2AC228F
:101E000000000000000000000000000000006F0063
:101E10004F012202E902A5035704FE049D05320684
:101E2000BF064407C1073808A80811097509D30976
:101E30002C0A800ACF0A190B600BA20BE10B1C0CB9
:101E4000540C890CBB0CEA0C160D400D680D8D0D61
:101E5000B00DD20DF10D1C8C548C898CBB8CEA8C8E
:101E6000168D408D688D8D8DB08DD28DF18D0F8E3C
:101E70002B8E458E5E8E768E8C8EA18EB48EC78E06
:101E8000D98EE98EF98E088F168F238F308F3B8F76
:101E9000468F518F5B8F648F6D8F758F7D8F848F91
:0A1EA0008B8F928F988F9E8FA48F76
:041D00004084C80C47
:101F00000063B4BEE36BD80973A4D1DE88D5014F5A
:101F10008EC7E09A8A396D6EB7E7A1C40467B69B95
:101F2000EBA3C102E0007601FF00135660BCEAE0BB
:101F3000DF3345A2A2E6BCE12E5579AAE3B2E663FF
:101F400000FFAFDA56EC6300FF8AE67FED0551A88B
:101F5000BEEA74C814557EA4E33FD6474298B0DA6F
:101F600078E80191A7A5DE7CDD45428BB3DD97DAE9
:101F70003BA80C9DDD48D73A9D148FE433C2387FCF
:101F80006E89DAFFE613AF1899D809000AA64487CC
:101F9000EE8E49166F00B3E63AD71760009EE55102
:101FA000CC197F00B1E43FE21D4F2CB1E437E71EAE
:101FB0004B15AFE453EA28393BBBE740ED2E70AE3A
:0B1FC000487601320A653496EB12DF10
:00000001FF
